:100000000AC018951895189518951895189518956B
:100010001895189518958FED8DBFC0ECE8EB4E2E16
:10002000DD275D2EEEE7F0E0A0E6B0E088278D93B7
:100030003197E9F7E3D266248FE087BB8FEF81BB6E
:1000400080E082BB8FE788BB84E690E04BD38CE0F6
:100050001DD3BF98A6E69C9197FF04C0B7990EC028
:100060009F779C93B79B0AC088E29F9399273AD3C6
:100070009F91B79B03C090689C934FD2A5D2EAE5AD
:10008000F7E09AD2E2E0F0E0B0D29CD2EAE6F7E004
:1000900093D2E4E0F0E0A9D2939A84E690E022D3F0
:1000A000939884E690E01ED380E080936400A1E6FC
:1000B0002CD380E08093630080E08093650084D23D
:1000C000EAE7F7E079D2C09AC39881E080936000B4
:1000D000BE98A6E69C9196FF04C0B69B0EC09F7B7F
:1000E0009C93B6990AC088E29F939927FBD29F916F
:1000F000B69903C090649C9313D182E08093600012
:10010000BD98A6E69C9195FF04C0B59B0EC09F7D4F
:100110009C93B5990AC088E29F939927E3D29F9157
:10012000B59903C090629C93FBD083E080936000FC
:10013000BC98A6E69C9194FF04C0B49B0EC09F7E21
:100140009C93B4990AC088E29F939927CBD29F9140
:10015000B49903C090619C93E3D0C39AC29884E0A1
:1001600080936000BE98A6E69C9196FF04C0B69B63
:100170000EC09F7B9C93B6990AC088E29F939927F3
:10018000B1D29F91B69903C090649C93C9D085E089
:1001900080936000BD98A6E69C9195FF04C0B59B36
:1001A0000EC09F7D9C93B5990AC088E29F939927C2
:1001B00099D29F91B59903C090629C93B1D086E08B
:1001C00080936000BC98A6E69C9194FF04C0B49B09
:1001D0000EC09F7E9C93B4990AC088E29F93992792
:1001E00081D29F91B49903C090619C9399D0C29A97
:1001F000C19887E080936000BE98A6E69C9196FF28
:1002000004C0B69B0EC09F7B9C93B6990AC088E23F
:100210009F93992767D29F91B69903C090649C934E
:100220007FD088E080936000BD98A6E69C9195FF02
:1002300004C0B59B0EC09F7D9C93B5990AC088E20F
:100240009F9399274FD29F91B59903C090629C9339
:1002500067D089E080936000BC98A6E69C9194FFEB
:1002600004C0B49B0EC09F7E9C93B4990AC088E2E0
:100270009F93992737D29F91B49903C090619C9323
:100280004FD0C19AC0988BE080936000BE98A6E6DC
:100290009C9196FF04C0B69B0EC09F7B9C93B69921
:1002A0000AC088E29F9399271DD29F91B69903C0F7
:1002B00090649C9335D08AE080936000BD98A6E658
:1002C0009C9195FF04C0B59B0EC09F7D9C93B599F2
:1002D0000AC088E29F93992705D29F91B59903C0E0
:1002E00090629C931DD08CE080936000BC98A6E641
:1002F0009C9194FF04C0B49B0EC09F7E9C93B499C4
:100300000AC088E29F939927EDD19F91B49903C0C9
:1003100090619C9305D08AE090E0E4D1D4CE94CE55
:10032000939A84E690E0DED1939884E690E0DAD167
:1003300000916400013009F001C048C000916400E0
:10034000023009F001C067C0009160000B3009F075
:100350002AC0A6E30C9104FB81E00EF480E08F93A9
:10036000A6E30C9105FB81E00EF480E09F91892BC0
:100370008F93A6E30C9106FB81E00EF480E09F9141
:10038000892B882309F401C0E4CF1ED1E8E8F7E007
:1003900013D1A4E68C918F5F8C9380E080936300EF
:1003A0008FE788BB90CE009160000C3009F00DC043
:1003B000EAE0F0E0A4E1C9D1A1E60D911C91041797
:1003C000150709F001C091C069C03AC000916000F2
:1003D0000C3009F01FC0EAE0F0E0A4E1B6D1A1E6DC
:1003E0000D911C910417150709F401C057C0A1E62F
:1003F0008CD180E08093630080E080936500A4E668
:100400008C918F5F8C93E0D0E8E9F7E0D5D08FE74F
:1004100088BB59CE15C0009160000C3009F010C0A7
:10042000EAE0F0E0A1E67BE77FD1CED0E8EAF7E0B2
:10043000C3D04AD0E2E0F0E0D8D08FE788BB34CE1A
:10044000A3E68C918F5F8C930091630046E0040FCC
:10045000A5E60C938FEBA5E61C91C5D0E8EBF7E081
:10046000ABD000916300043010F009F001C001C06E
:1004700015C0A1E60D911C914AE050E08AD0A1E69A
:100480000D931C93A1E60D911C91A0E64D9155276B
:10049000040F151FA1E60D931C93089595D0EAEB68
:1004A000F7E08AD084E690E01DD1939AE3E0F0E093
:1004B0009CD0939887D0EAE5F7E07ED0E4E1F0E0C5
:1004C00094D08FE788BBF0CD84E690E00BD1939A6F
:1004D00088EC90E007D1939888EC90E003D1939A50
:1004E00088EC90E0FFD0939808956ED0E8EAF7E0AA
:1004F00063D0EADF67D0E8ECF7E05ED08CE291E011
:10050000F1D08FE788BB949AE1E0F0E06ED0949848
:100510005BD0E1E0F0E069D0C7CDE1E0F0E065D08C
:10052000B79901C014C0EAE0F0E002ED14E0A0E1E8
:10053000BB277BE7F9D0C8DF47D0E6EDF7E03CD03A
:1005400041D0E6EEF7E038D0E4E0F0E04ED0ACCDBC
:1005500004D01FD000FC0CD008950024E89457FF6D
:1005600002C009D0689400F80BD010F80124089557
:1005700002D009D00895509540954F5F5F4F089580
:10058000E89417FF0895009510950F5F1F4F68942A
:100590000895752F642F55274427FF93F1E1889420
:1005A00005C010F4460F571F5695479517950795A8
:1005B000FA95B9F7FF910895A4D0802D11F060D07D
:1005C000FBCF089580EC62C081E060D014D080E859
:1005D0005DC08FE7213039F08FEB223021F08FE8BA
:1005E000233009F08FEC810F51C088EE93E07AD070
:1005F0003197D9F7089583E0992774C08AEF90E086
:1006000071D0BB9ABA9AB99AB89A8E9A8D9A9598DF
:1006100085E090E067D09698C398C298C19AC09A36
:10062000969AEF93FF93E0E6F0E050D0FF91EF91C0
:10063000969855D0969AEF93FF93E0E6F0E046D077
:10064000FF91EF9196984BD0969AEF93FF93E0E647
:10065000F0E03CD0FF91EF91969841D0C098969AE7
:10066000EF93FF93E0E6F0E031D0FF91EF919698A1
:1006700036D088E20BD08EE009D086E007D008950E
:10068000959A829505D004D02AD008959598F9CFEF
:10069000859510F4C09A01C0C098859510F4C19A50
:1006A00001C0C198859510F4C29A01C0C298859581
:1006B00010F4C39A01C0C398969AEF93FF93E0E6B3
:1006C000F0E004D0FF91EF91969808953197F1F7FB
:1006D0000895689462F80895E89462F8089581E0B6
:1006E00090E000C0EF93FF93EE27E82BE92B31F069
:1006F000E8EEF3E03197F1F70197D1F7FF91EF9131
:100700000895C89531960020089582E001C084E0E4
:1007100099279D938A95E9F70895E199FECFEEBB5D
:100720003196089591E001C092E07B3751F47FB794
:10073000F894F3DF8D918DBBE29AE19A9A95C9F70F
:100740007FBF7727089591E001C092E0E6DFE09A4D
:100750008DB38D939A95D1F708955757572E4156DB
:10076000522E344D472E434F4D002020436F646579
:100770004C6F636B415652202000202020456E7440
:10078000657220636F64650020456E746572206F2A
:100790006C6420636F64650020456E746572206E22
:1007A000657720636F64650020436F646520616333
:1007B00063657074656400002A00202020436F6424
:1007C000652077726F6E670020202020556E6C6F59
:1007D000636B656400002020496E697469616C2058
:1007E000636F646500002020202020697320202092
:0607F00031323334000039
:00000001FF
